:1000000012C02CC02BC02AC029C028C027C026C0BF
:1000100025C024C023C022C021C020C01FC01EC0D4
:100020001DC01CC01BC011241FBECFE5D4E0DEBF25
:10003000CDBF10E0A0E6B0E0ECE5F2E002C0059034
:100040000D92A037B107D9F710E0A0E7B0E001C0EA
:100050001D92A037B107E1F731D0FFC0D1CF0F9388
:100060001F9388EA91E60197F1F781B38F6381BB13
:1000700082B3807E836082BB55D002EE14E0C8015B
:100080000197F1F788E274D0C8010197F1F788E28F
:100090006FD0C8010197F1F78CE06AD0C8010197D1
:1000A000F1F781E065D0C8010197F1F786E060D0F3
:1000B000C8010197F1F71F910F910895CF93DF9336
:1000C000CEDF20E137E289E190E00197F1F721509E
:1000D0003040C9F780E84CD080E690E056D080EC04
:1000E00047D086E690E051D040E050E018C089E16A
:1000F00090E00197F1F721503040C9F74F5F5F4F13
:100100004230510561F43AD0C0E0D0E09E01205D5C
:10011000822F31D02196CA30D105C4F3F5CF20E12A
:1001200037E2E5CF959A83E08A95F1F7959808959F
:100130000F931F93082F82B3902F92959F70807F0B
:10014000982B92BB11E0812F8A95F1F7EBDF82B3F8
:100150000F70807F802B82BB1A95F1F7E3DF84E17B
:100160008A95F1F782B3807F82BB1F910F9108952A
:100170009498DEDF0895949ADBDF089581E0F8DF3C
:1001800082EE94E00197F1F70895CF93DF93EC01AD
:1001900002C0F1DF219688818823D9F7DF91CF91C2
:1001A0000895CF93DF93EC01DE014FD0802D88239B
:1001B00019F0E1DF2196F8CFDF91CF910895CF9329
:1001C000DF93CDB7DEB722970FB6F894DEBF0FBE30
:1001D000CDBF81B38F6381BB8CE49DE10197F1F7C3
:1001E00082B3807E836082BB9DDF82EE94E00197C4
:1001F000F1F798DF8AEF90E0FC013197F1F79A83ED
:10020000898390DF89819A81FC013197F1F722B3CC
:10021000207E226022BBFC013197F1F79A8389830B
:1002200081DF89819A810197F1F788E2A1DF8CE073
:100230009FDF86E09DDFA2DF22960FB6F894DEBF37
:100240000FBECDBFDF91CF910895E199FECFBFBB27
:0C025000AEBBE09A11960DB20895FFCFEE
:10025C0048616C6C6F0053616C7661746F726500F1
:00000001FF
